:020000040000FA
:040000006400682907
:08000800F1000308F20083017E
:100010008C10A30A2B082302031D1F28A30101082B
:10002000A6008101260803191D28250A26020319A6
:100030001F282503260203191F282608A5000008EB
:100040007F3AA40025080319A417F8308505240871
:1000500086002030040239208504840A23300402FB
:10006000031D34282030840072088300F10E710EC5
:1000700009000339820701340234043400340F3993
:1000800082073F3406345B344F3466346D347D343C
:1000900027347F346F3400347F3440347F3400346D
:1000A00063346400271CAF202718A1205820512852
:1000B000AD0A06302D02031D0800AD01AC0A7F30E9
:1000C0002C0203197228FF302C0203197B28000030
:1000D0000000000000000000000000000000000020
:1000E0000000080005082839AE00000000000000EC
:1000F000000000000800050828392E06031D08002E
:10010000AE1D8C28AE1E9428A710271C0800AF0B2C
:1001100008002710FA200800271C9C28A7180800B0
:10012000AB0A2930AF000800271C9C28A71808003C
:10013000AB032930AF0008002714A7142930AF0003
:1001400008002B08D52029083F20A0002A0E0F39CF
:100150003F20A1002A080F393F20A20008002508EF
:10016000D5202908031DC9282A0E0F39031DBF28D1
:10017000A001A1012A080F393F20A2000800A00118
:100180002A0E0F393F20A1002A080F393F20A20074
:10019000080029083F20A0002A0E0F393F20A100A7
:1001A0002A080F393F20A2000800A800A901280E44
:1001B00028070F398318163E8318063E063E831C17
:1001C000FA3E281A1B3E831CFA3EA81A303E281B12
:1001D000603EA81B203E603EA90D291CA03EAA003F
:1001E000A81BA90A080083169B011C141A08831275
:1001F000AB00080083169B011C141A0883122B06FF
:10020000031908002B0883169A009B011C158B13F9
:1002100055309D00AA309D009C148B1764009C18DB
:100220000F291C11831208004400490047004900AF
:10023000540041004C002000530050004500450090
:1002400044004F004D00450054004500520020007E
:100250002800430029003200300031003100200026
:100260004D0041004D004500440020002000680082
:100270007400740070003A002F002F0065006C00BD
:1002800065006300740072006F0061007600740006
:100290006F002E006E00610072006F0064002E007F
:1002A00072007500203420344934443443344F34D0
:1002B000443445343A3420343934303439343434E5
:1002C0003334373436343534303432342034203417
:1002D00007309F00850186018316F83085000030C5
:1002E0008600BA308100F93092008C1483126400C9
:1002F00020308400EF178001840AEF1B7B29640003
:1003000020308400F3207C3092000B178B1751288B
:02400E00053F6C
:02420000960026
:00000001FF
